:020000040000FA
:06000000DDEF13F0120019
:0600080004EF08F01200F5
:060018000CEF08F01200DD
:06100000DDEF13F0120009
:0610080011EF12F01200CE
:0610180046EF12F0120089
:06102A000100E6270000B2
:08103000600000003C0000001C
:08103800D9CFE6FFE1CFD9FF9B
:10104000E6526A6A686A9F0E6B6EFB0E696E6D8C63
:101050006D9C6E6A020EE66EE66AE66A710EE66ED8
:101060000F0EE66EC3EC13F00B6E050EE15E0B5037
:10107000DF6ADF500B6E0C6A100E0B5C000E0C5812
:1010800010E2DF50040DF3CFE9FFF4CFEAFF000ECA
:10109000E926040EEA22EE6AEE6AEE6AEE6ADF2ABA
:1010A000E8D7160E706E68A60CD0030EE66E680EBA
:1010B000E66E0F0EE66ECDEC0FF0E552E552E5520E
:1010C000F2D70001B76BBC6BBD6BBE6B6D98080EA1
:1010D000AB6F040EAC6F9D6B9C6BE552E552E7CF96
:1010E000D9FF1200D9CFE6FFE1CFD9FFE6520001C8
:1010F0009C5111E105D06D6A696A00019C6B86D034
:101100006D6A696A6DB602D06D86FCD70001010E6A
:101110009C6F160E6F6E9C0508E16DBA06D0686A6A
:10112000696A69806988020E9C6F6850040B04E04C
:101130006950040B01E0A1D86DB268D06850010B72
:1011400011E06950010B0EE077DF0001040E9C6F87
:101150000401400E026F040E036F080E016F006B56
:101160008C0E00136850100B0FE06950100B0CE050
:1011700075D8040EE66E680EE66E0F0EE66ECDECC8
:101180000FF0E552E552E5526850400B10E069500F
:10119000400B0DE0DAEC12F0060EE66E680EE66E1D
:1011A0000F0EE66ECDEC0FF0E552E552E5526850B9
:1011B000200B04E06950200B01E02DD86850020B91
:1011C00006E06950020B03E0DBEC12F06A6A040EE1
:1011D00000019C5D01E21AD069A618D0DF6A040EF6
:1011E000DF5C14E268A60FD06CCFC4F0030EE66E8D
:1011F000680EE66E0F0EE66ECDEC0FF0E552E5528E
:10120000E5524ED801D002D0DF2AE9D7E552E552A7
:10121000E7CFD9FF120070A015D09FC0E9FFA0C092
:10122000EAFFEF5080080DE1ABC0E9FFACC0EAFF78
:10123000EF50840806E19FC0E9FFA0C0EAFF8C0ED2
:10124000EF6E7090050EE66E680EE66E0F0EE66E9F
:10125000CDEC0FF0E552E552E55212006984040E20
:10126000E66E680EE66E0F0EE66ECDEC0FF0E55200
:10127000E552E5526D82D8EF12F06D92D9EC12F082
:10128000699468A40CD0020EE66E680EE66E0F0E2E
:10129000E66ECDEC0FF0E552E552E552F2D71200C2
:1012A000FD0E0001C41520E17E0EC415E8407F0B41
:1012B000040DF3CF9FF0F4CFA0F0000E9F27040E93
:1012C000A0239FC0A1F0A0C0A2F0A1759FC0E9FF1C
:1012D000A0C0EAFFEF503C0BE842E8420D0802E1F3
:1012E00009D801D01ED805D0FD0EC415040801E1AF
:1012F00020D81200ABC0E9FFACC0EAFFEF50800B72
:1013000005E0ABC0E9FFACC0EAFFEF6A0001B36BD8
:10131000B46BB86BB96BB76BF7D8DCEC12F024EF99
:101320000CF0020E0001B45D02E1EBDB01D04ED8FF
:101330001200D9CFE6FFE1CFD9FFE652ABC0E9FFFB
:10134000ACC0EAFFEF50400B01E0010EDF6E000180
:10135000AB75080E9C5D0AE142C46EFF6E5000083A
:1013600003E2100E9C6F02D0040E9C6FB40528E1BE
:10137000ABC0E9FFACC0EAFF020EE926000EEA228C
:10138000480EEE6E040EED6E31DB020E0001B35D11
:1013900007E1ABC0E9FFACC0EAFF840EEF6E0FD0EF
:1013A000DF5007E1ABC0E9FFACC0EAFFC80EEF6E4B
:1013B00006D0ABC0E9FFACC0EAFF880EEF6E01D0EB
:1013C00005D8E552E552E7CFD9FF1200D9CFE6FFA5
:1013D000E1CFD9FF030EE126020E0001B45D4AE120
:1013E0006D50100B47E09FC0E9FFA0C0EAFFEE522E
:1013F000EF500B6E0C6A080E0B1801E10C503AE12D
:101400009FC0E9FFA0C0EAFFEF503C0BE842E84272
:101410000D0830E1A1C0E9FFA2C0EAFFEF50800B48
:1014200029E1A1C0E9FFA2C0EAFF020EE926000EF1
:10143000EA22400EEE6E040EED6EDF6ADF500B6E98
:101440000C6A080E0B5C000E0C5813E2DF50EA6ABF
:10145000480FE96E040EEA22EF50E66EDF50EA6AAA
:10146000400FE96E040EEA22E552E750EF6EDF2AE4
:10147000E5D731D0B46BA1C0E9FFA2C0EAFFEE52BC
:10148000080EEF6EA1C0E9FFA2C0EAFF020EE92636
:10149000000EEA22400EEE6E040EED6EA1C0E9FFD2
:1014A000A2C0EAFF8C0EEF6EABC0E9FFACC0EAFF52
:1014B000EF6A040EAB190B6EACC00CF0010E0BC042
:1014C000DBFF020E0CC0DBFF010EDBCFE9FF020EDB
:1014D000DBCFEAFFEF6A0001BCAF0CD0BF51C011F7
:1014E00007E005D0C0C0FAFF0001BF51F96EFADF76
:1014F0000001BC9F030EE15C02E2E16AE552E16E8D
:10150000E552E7CFD9FF120004014051600BE842D9
:10151000E842E842E842E842000901E04CD041518B
:101520000C0A48E00B0A43E00C0A35E0010A26E009
:101530000B0A22E0020A20E0030A1CE0080A10E07D
:10154000010A0CE00F0A08E0030A01E033D00001B1
:10155000B78F080E9C6F2FD0BCD82DD063DB2BD05B
:1015600000019D0EB56F000EB66FB781010EB86F0A
:10157000B78F21D008D91FD01FD81DD044510001EA
:10158000B56FB66B9E0EB527000EB623B781010E60
:10159000B86FB78F10D00001B78F04014451EA6AC9
:1015A0009E0FE96E000EEA2242C4EFFF04D0DEEC8B
:1015B00012F001D000D01200D9CFE6FFE1CFD9FF61
:1015C000040EE1260401420510E140511F0B000901
:1015D0000CE10001B78F030E0401415D04E100013D
:1015E000010EC36F02D00001C36B0401425167E1D9
:1015F00040511F0B020863E144510F0B00095FE0EB
:101600000001B78F040144BF10D044510F0BE96EA5
:10161000EA6AD890E936EA36A30EE926000EEA22F5
:10162000EECFDEFFEDCFDDFF0FD044510F0BE96EA3
:10163000EA6AD890E936EA36AB0EE926000EEA22CD
:10164000EECFDEFFEDCFDDFF030E415D07E1DECF24
:10165000E9FFDDCFEAFF840EEF6E31D044510F0B6E
:101660000C6A700F0B6E0F0E0C22020E0BC0DBFF0C
:10167000030E0CC0DBFF020EDBCFE9FF030EDBCF56
:10168000EAFFEE90ED5244AF0DD0DECFE9FFDDCFA3
:10169000EAFFEF6ADF74DECFE9FFDDCFEAFF400E3D
:1016A000EF6E0DD0DECFE9FFDDCFEAFF880EEF6EE3
:1016B000DF74DECFE9FFDDCFEAFFC80EEF6E040E68
:1016C000E15C02E2E16AE552E16EE552E7CFD9FF63
:1016D0001200800E0401405D55E10001C00EB76F9D
:1016E00004014351030A2EE0010A0EE0030A03E05D
:1016F0000001B76B47D00001DE0EB56F250EB66F47
:10170000120EB86FB96B3ED04251F66EF76AD890A0
:10171000F636F7369F0EF626260EF7220900F5CF8D
:10172000B5F00A00F5CFB6F0020E0001F76AB52554
:10173000F66EB651F7220900F5CFB8F00A00F5CFE2
:10174000B9F020D0030E425D1AE24251F66EF76AFC
:10175000D890F636F736A10EF626260EF7220900A7
:10176000F5CFB5F00A00F5CFB6F0B5C0F6FFB6C0BC
:10177000F7FF0800F5500001B86FB96B02D0000107
:10178000B76B00D01200D9CFE6FFE1CFD9FF020E30
:10179000E1260401486B496B40511F0B020A12E01D
:1017A000030A0DE0010A01E03BD00001B78F0401FC
:1017B00048810001C30502E10401488331D00001E2
:1017C000B78F2ED00001B78F040144BF10D0445111
:1017D0000F0BE96EEA6AD890E936EA36A30EE926DD
:1017E000000EEA22EECFDEFFEDCFDDFF0FD0445139
:1017F0000F0BE96EEA6AD890E936EA36AB0EE926B5
:10180000000EEA22EECFDEFFEDCFDDFFDECFE9FFF7
:10181000DDCFEAFFEF50040B02E0010E486F00D06D
:101820000001B7AF07D0480EB56F040EB66FB78191
:10183000020EB86F020EE15C02E2E16AE552E16E6F
:10184000E552E7CFD9FF12006D980001B7BF4AD02B
:10185000BCAF28D0020EB46FABC0E9FFACC0EAFF4A
:10186000EE52EF6AABC0E9FFACC0EAFFC80EEF6E04
:10187000A1C0E9FFA2C0EAFFEE52080EEF6EA1C0C0
:10188000E9FFA2C0EAFF020EE926000EEA22480E96
:10189000EE6E040EED6EA1C0E9FFA2C0EAFFC80E15
:1018A000EF6E1FD0A1C0E9FFA2C0EAFFEE52080E02
:1018B000EF6EA1C0E9FFA2C0EAFF020EE926000E0A
:1018C000EA22400EEE6E040EED6EA1C0E9FFA2C04A
:1018D000EAFF8C0EEF6EABC0E9FFACC0EAFF840EEE
:1018E000EF6E83D0BCBF81D0040140AF56D0000161
:1018F000B8510401465D0001B9510401475904E2A1
:1019000046C4B8F047C4B9F071D80001010EB46FF5
:10191000A1C0E9FFA2C0EAFFEE52080EEF6EA1C01F
:10192000E9FFA2C0EAFF020EE926000EEA22400EFD
:10193000EE6E040EED6EA1C0E9FFA2C0EAFF800EBC
:10194000EF6E9FC0E9FFA0C0EAFFEE52080EEF6EF7
:101950009FC0E9FFA0C0EAFF020EE926000EEA22BE
:10196000400EEE6E040EED6E9FC0E9FFA0C0EAFFD0
:10197000800EEF6EABC0E9FFACC0EAFF020EE926B5
:10198000000EEA22480EEE6E040EED6EABC0E9FFCB
:10199000ACC0EAFFC80EEF6E28D00001020EB46F93
:1019A000ABC0E9FFACC0EAFFEE52EF6AABC0E9FFA3
:1019B000ACC0EAFFC80EEF6EA1C0E9FFA2C0EAFF0B
:1019C000EE52080EEF6EA1C0E9FFA2C0EAFF020EC0
:1019D000E926000EEA22480EEE6E040EED6EA1C05E
:1019E000E9FFA2C0EAFFC80EEF6E1200D9CFE6FFF2
:1019F000E1CFD9FF020EE1260001080EB85D000E0E
:101A0000B9590EE2B8C0DEFFB9C0DDFFB35103E142
:101A1000010EB36F04D0B30502E1020EB36F03D021
:101A2000080EDE6EDD6AABC0E9FFACC0EAFFEF92E4
:101A3000ABC0E9FFACC0EAFFEF90ABC0E9FFACC0C0
:101A4000EAFF010EDB50EF12ABC0E9FFACC0EAFFCA
:101A5000EE52DFCFEFFF000EDB50B85F010EDB5020
:101A6000B95B480EC16F040EC26FB7B121D0D9CF98
:101A7000E9FFDACFEAFFEE50ED1019E0B5C0F6FF4E
:101A8000B6C0F7FFB52B000EB6230800F550E66E82
:101A9000C1C0E9FFC2C0EAFFC12B000EC223E5525C
:101AA000E750EF6EDF06010E01E2DB06E0D71FD044
:101AB000D9CFE9FFDACFEAFFEE50ED1018E0B5C05C
:101AC000E9FFB6C0EAFFB52B000EB623EF50E66E75
:101AD000C1C0E9FFC2C0EAFFC12B000EC223E5521C
:101AE000E750EF6EDF06010E01E2DB06E1D7020EE2
:101AF000E15C02E2E16AE552E16EE552E7CFD9FF2F
:101B00001200D9CFE6FFE1CFD9FF020EE1269FC038
:101B1000E9FFA0C0EAFFEE52EFCFDFFFDFCF0BF00F
:101B20000B500001BD5D000EBE5903E2BDC0DFFFDA
:101B300009D0DF500B6E0C6A0B50BD5DBD6F0C50B1
:101B4000BE59BE6F010EDB6ADF50F36E010EDBCFB4
:101B5000F4FFF350F45C16E2010EDB50EA6A480F22
:101B6000E96E040EEA22EF50E66EBAC0E9FFBBC090
:101B7000EAFFBA2B000EBB23E552E750EF6E010ED1
:101B8000DB2AE2D7000ED880BD55000EBE5528E2F4
:101B9000A1C0E9FFA2C0EAFFEE52080EEF6EA1C09D
:101BA000E9FFA2C0EAFF020EE926000EEA22480E73
:101BB000EE6E040EED6E9FC0E9FFA0C0EAFFEF508D
:101BC000400B07E1A1C0E9FFA2C0EAFFC80EEF6E1B
:101BD00006D0A1C0E9FFA2C0EAFF880EEF6E18D0C0
:101BE000A1C0E9FFA2C0EAFF020EE926000EEA2228
:101BF000400EEE6E040EED6EBF51C01107E005D031
:101C0000C0C0FAFF0001BF51F96EFADF0001BC9FAE
:101C1000020EE15C02E2E16AE552E16EE552E7CFD5
:101C2000D9FF12000001B78F020EE66EE66AE66A7F
:101C3000710EE66E0F0EE66EC3EC13F00B6E050E22
:101C4000E15E0B50010EE66EE66AE66A9E0EE66EF7
:101C5000000EE66EC3EC13F00B6E050EE15E0B504A
:101C600042C49DF00401425104E10001100E9C6F3A
:101C700005D00001200E9C6FDFEC12F01200D9CFCE
:101C8000E6FFE1CFD9FF020EE126000EDE6E040E64
:101C9000DD6EFD0EDB50E8240D6EFE0EDB50040DF4
:101CA000F3500D24040DF3500B6E0C6A020E0F0B53
:101CB00005E0D8900C320B32E806FBE1D8900B36E9
:101CC0000C36D8900B360C36D9CFE9FFDACFEAFFC5
:101CD0000B50EE260C50ED22DECFE9FFDDCFEAFF00
:101CE000EF9EFD0EDB500FE1FE0EEA6ADB34FE0BC9
:101CF000EA36E96EA30EE926000EEA22DECFEEFFF9
:101D0000DDCFEDFF0ED0FE0EEA6ADB34FE0BEA36C5
:101D1000E96EAB0EE926000EEA22DECFEEFFDDCF44
:101D2000EDFFDECFE9FFDDCFEAFFEF9CDECFE9FF7D
:101D3000DDCFEAFF040EE926000EEA22EF8C020E48
:101D4000E15C02E2E16AE552E16EE552E7CFD9FFDC
:101D50001200D9CFE6FFE1CFD9FF020EE126FE0E39
:101D6000DB500C6A700F0B6E0F0E0C220BC0DEFFE7
:101D70000CC0DDFFFD0EDB50E66EDECFE9FFDDCFF0
:101D8000EAFFE552E750EE6EED6AFD0EDBA407D0E8
:101D9000E66AFE0EDBCFE6FF72DFE552E552FD0E8E
:101DA000DBA208D0010EE66EFE0EDBCFE6FF67DF9A
:101DB000E552E552020EE15C02E2E16AE552E16EB3
:101DC000E552E7CFD9FF1200D9CFE6FFE1CFD9FF27
:101DD000020EE126FE0EDB5020E1A1C0E9FFA2C009
:101DE000EAFFEE52080EEF6EA1C0E9FFA2C0EAFFC3
:101DF000020EE926000EEA22400EEE6E040EED6E93
:101E0000A1C0E9FFA2C0EAFF8C0EEF6EABC0E9FFF4
:101E1000ACC0EAFF840EEF6E3DD0FD0EDB50E8242F
:101E20000D6EFE0EDB50040DF3500D24040DF3CFA8
:101E30000BF0F4CF0CF0000E0B26040E0C220BC09E
:101E4000DEFF0CC0DDFF840E0B6EDECFE9FFDDCFC1
:101E5000EAFF0B50EF12FD0EDB50E8240D6EFE0E74
:101E6000DB50040DF3500D24010F040DF3CF0BF0E4
:101E7000F4CF0CF0000E0B26040E0C220BC0DEFF7C
:101E80000CC0DDFF840E0B6EDECFE9FFDDCFEAFF75
:101E90000B50EF12020EE15C02E2E16AE552E16EE4
:101EA000E552E7CFD9FF1200D9CFE6FFE1CFD9FF46
:101EB000020EE126FD0EDB500FE0FE0EEA6ADB3477
:101EC000FE0BEA36E96EAB0EE926000EEA22EECFF3
:101ED000DEFFEDCFDDFF0ED0FE0EEA6ADB34FE0B37
:101EE000EA36E96EA30EE926000EEA22EECFDEFF07
:101EF000EDCFDDFFDECFE9FFDDCFEAFF020EE92601
:101F0000000EEA22FB0EDBCFEEFFFC0EDBCFEDFF77
:101F1000DECFE9FFDDCFEAFFEE52FA0EDBCFEFFFB7
:101F2000400E0B6EDECFE9FFDDCFEAFF0B50EF1660
:101F3000880E0B6EDECFE9FFDDCFEAFF0B50EF120C
:101F4000FD0EDB500CE0FE0EEA6ADB34FE0BEA36D7
:101F5000E96EAB0EE926000EEA22EF740BD0FE0EFE
:101F6000EA6ADB34FE0BEA36E96EA30EE926000EC0
:101F7000EA22EF74DECF0BF0DDCF0CF00BC0F3FFE5
:101F80000CC0F4FF020EE15C03E200D0E16AE5520E
:101F9000E16EE552E7CFD9FF1200D9CFE6FFE1CFDE
:101FA000D9FF010EF36EFC0EDB5004E0D890F3363F
:101FB000E806FCE1F350E81C0B6EFD0EDBCFE9FFF9
:101FC000FE0EDBCFEAFF0B50EF16E552E7CFD9FF4D
:021FD0001200FD
:0E1FD200040140511F0B010801E04AD04051AC
:101FE000600BE842E842E842E842E842010801E0CA
:101FF00040D0445103E0440501E03BD04151220A66
:1020000033E0030A26E0010A17E0210A0EE0010A84
:1020100001E02FD00001F20EB56F010EB66F080E71
:10202000B86FB96BB781B78F24D00001F20EB56FCE
:10203000010EB66FB78F1DD046C4BDF047C4BEF0C9
:102040000001880EBA6F050EBB6FBF6BC06BBC8FF3
:1020500010D00001880EB56F050EB66F070EB86F71
:10206000B96BC10EB76F05D042C4EDF10001B78F57
:1020700000D012000501886B4B0E896F8A6B8B6B49
:102080008C6B8D6B080E8E6F0101E26BE16B1A0E8B
:10209000E66E020EE66EA9EC0EF0E552E5521E0E5B
:1020A000E66E030EE66EA9EC0EF0E552E552400E28
:1020B000E66E080EE66E050EE66EE66A030EE66E46
:1020C00054EC0FF00B6E050EE15E0B50F3CFE9F10F
:1020D000F4CFEAF10101EB6BEC6B1200D9CFE6FF14
:1020E000E1CFD9FF0101E16BE951EA1102E1000EF4
:1020F00008D0E9C1E9FFEAC1EAFFEF50800B01E037
:10210000010E000945E1FC0EDBCF0BF0E9C1E9FF50
:10211000EAC1EAFFEE52EF50D8800B5408E2E9C161
:10212000E9FFEAC1EAFFEE52FC0EEFCFDBFFE16B05
:10213000FC0EDB50E15D19E2E151EA6A080FE96E3D
:10214000050EEA22EF50E66EE151E76EFD0EDBCFA1
:10215000E9FFFE0EDBCFEAFFE750E926000EEA2298
:10216000E552E750EF6EE12BE3D7400EE66E080E26
:10217000E66E050EE66EE66A030EE66E54EC0FF0B0
:102180000B6E050EE15E0B50F3CFE9F1F4CFEAF1EF
:102190000101E15100D0E552E7CFD9FF1200D9CFBC
:1021A000E6FFE1CFD9FF0101E2510CE1FD0EDBCFEB
:1021B000E3F1FE0EDBCFE4F1FC0EDBCFE7F1010E25
:1021C000E86FE26FE552E7CFD9FF1200D9CFE6FF03
:1021D000E1CFD9FF030EE1260101E25101E02ED04B
:1021E000DF6AFD0EDBCF06F0FE0EDBCF07F0DE521E
:1021F00006C0DEFF07C0DDFFDD52DF2ADF500B6EB9
:102200000C6AFF0E0B1801E10C5001E10BD0010E1E
:10221000DBCFE9FFDB2A020EDBCFEAFF01E3DB2A9B
:10222000EF50EBE1FD0EDBCFE3F1FE0EDBCFE4F18F
:10223000DFCFE7F10101010EE86FE26F030EE15C11
:1022400002E2E16AE552E16EE552E7CFD9FF120002
:10225000D9CFE6FFE1CFD9FF030EE1260101E2511C
:1022600001E02FD0DF6AFD0EDBCF06F0FE0EDBCFE4
:1022700007F0DE5206C0DEFF07C0DDFFDD52DF2AB9
:10228000DF500B6E0C6AFF0E0B1801E10C5001E1E0
:102290000CD0010EDBCFF6FFDB2A020EDBCFF7FFFF
:1022A00001E3DB2A0800F550EAE1FD0EDBCFE3F1A4
:1022B000FE0EDBCFE4F1DFCFE7F10101E86B010EA9
:1022C000E26F030EE15C02E2E16AE552E16EE55283
:1022D000E7CFD9FF1200D9CFE6FFE1CFD9FF020E39
:1022E000E1260101EB51EC1102E1000E08D0EBC137
:1022F000E9FFECC1EAFFEF50800B01E0010E00099D
:1023000001E085D0030EE25D01E1E26BE25101E103
:102310007ED0020EE25D16E1E66A000EE66EE66A27
:10232000010EE66E030EE66E54EC0FF00B6E050E1A
:10233000E15E0B50F3CFEBF1F4CFECF10101030EB2
:10234000E26F65D0E20563E1400E0B6E0C6AE75167
:102350000B5C000E0C5803E2400EDF6E02D0E7C1AA
:10236000DFFFDF50E75DE76F480EE56F050EE66FB4
:10237000010EDFCFDBFFE85117E1010EDB5013E068
:10238000E3C1F6FFE4C1F7FF0800F550E5C1E9FF3E
:10239000E6C1EAFFEF6EE52B000EE623E32BE42314
:1023A000010EDB06EAD715D0010EDB5012E0E3C1C7
:1023B000E9FFE4C1EAFFEF50E5C1E9FFE6C1EAFF4A
:1023C000EF6EE52B000EE623E32BE423010EDB0684
:1023D000EBD7E75108E1400EDF5C03E1020EE26F4C
:1023E00002D0030EE26FDFCFE6FF480EE66E050E69
:1023F000E66E010EE66E030EE66E54EC0FF00B6E09
:10240000050EE15E0B50F3CFEBF1F4CFECF1020ED1
:10241000E15C02E2E16AE552E16EE552E7CFD9FF05
:022420001200A8
:0E242200DACFE4FFE2CFDAFFE9CFE4FFEACF42
:10243000E4FFE652F2A222D000019B6B818899C092
:10244000E9FFEA6AE9BEEA68800EE926010EEA229F
:1024500083CFEFFF992B9A51E76E9919E8AE02D01E
:10246000993503D0E750D880995505E2010E976F52
:10247000986B819601D081989B6BF292E552E5CFE3
:10248000EAFFE5CFE9FFE5CFDAFF1100D8CFE4FF9F
:10249000E0CFE4FFE46EDACFE4FFE2CFDAFFE6520A
:1024A000F2A41ED0817200019B2B020EE76E9B19D5
:1024B000E8AE02D09B3503D0E750D8809B550FE2A1
:1024C000000EE76E9919E8AE02D0993503D0E750B7
:1024D000D880995504E2010E976F986B9B6BF2942C
:1024E000E552E5CFDAFFE550E5CFE0FFE5CFD8FFD5
:1024F0001000FC0EE66EA3EC13F0E552D76AD66A24
:10250000850ED56E200EF26EF292F294F194F28A5C
:10251000F288D08EF28EF28C120012D8010E936ED9
:10252000F00E946E9568E5DF8192819481868198A2
:102530000001976B986B72EC08F006D8FCD712007C
:102540000F0EC1121CEF08F0D9CFE6FFE1CFD9FF83
:10255000E652200E00019C5D03E36D50020B01E08A
:1025600022D0000197051DE19B6B0101E25118E1AA
:102570008194000198510FE10101800EE36F010E7B
:10258000E46F99C0E7F10101010EE86F0101E26F0C
:102590000001986F04D0976B8186996B819801D068
:1025A00081846BEC11F0E552E552E7CFD9FF1200C0
:1025B0001200120012001200E9EF0FF012003AEFC1
:1025C00010F06D840101080EDF6F070EE06FDF076A
:0E25D000000EE05BDF51E011FAE16D941200A5
:0225DE001201E8
:1025E000000202000008D8040A00010001020001F4
:1025F00009024300020100C0320904000001020286
:102600000100052400100104240202052406000133
:1026100005240100010705820308000209040100E6
:10262000020A0000000705030240000007058302BC
:102630004000000403090434034D00690063007284
:10264000006F00630068006900700020005400659E
:1026500000630068006E006F006C006F0067007917
:1026600000200049006E0063002E00340343004444
:102670000043002000520053002D0032003300328E
:1026800000200045006D0075006C00610074006959
:10269000006F006E002000440065006D006F00F0C8
:0726A00025332637266B26C7
:0826A8002A0EF66E100EF76E0B
:1026B000000EF86E00010900F550D66F0900F550C4
:1026C000D76F03E1D66701D03DD00900F550D16F37
:1026D0000900F550D26F0900F550D36F09000900C9
:1026E000F550E96E0900F550EA6E0900090009008D
:1026F000F550D46F0900F550D56F09000900F6CFE9
:10270000D8F0F7CFD9F0F8CFDAF0D1C0F6FFD2C0C9
:10271000F7FFD3C0F8FF0001D45302E1D55307E01F
:102720000900F550EE6ED407F8E2D507F9D7D8C006
:10273000F6FFD9C0F7FFDAC0F8FF0001D607000E98
:06274000D75BBFD71200B9
:0A274600D9CFE6FFDACFE6FFE1CFBE
:10275000D9FFE2CFDAFFF292FD0EDBA202D0F18CBC
:1027600001D0F19CDBA002D0F18E01D0F19E9380CC
:10277000DBAE02D0F28801D0F298E552E5CFDAFF65
:06278000E7CFD9FF1200B3
:0A278600FE0EE3CFE9FFFF0EE3CFE4
:10279000EAFFE9CFF3FFEACFF4FFFB0EE35003E1DA
:1027A000FC0EE35009E0FB0EE30602E2FC0EE3063A
:0A27B000FD0EE350EE6EF1D71200AB
:0627BA0013EE00F023EE17
:1027C00000F0F86A0A9C54EC13F0F2EC13F08DEC74
:0627D00012F0FBD712001D
:0A27D60000EE00F00F0EEE6AEA625A
:0427E000FDD712000F
:0227E4001200E1
:0A27E6004142434445464748494C30
:1027F0004D4E4F505152535455565A303132333456
:1028000035363738394142434445464748494C4DAF
:102810004E4F505152535455565A0D0A0000000065
:022820003F0077
:020000040030CA
:0100000024DB
:010001000EF0
:0100020038C5
:010003001EDE
:010005008179
:010006008178
:010008000FE8
:01000900C036
:01000A000FE6
:01000B00E014
:01000C000FE4
:01000D0040B2
:00000001FF
